S00C00006D61696E2E7372656373
S11300000C942A000C9445000C9445000C94450073
S11300100C9445000C9445000C9445000C94450048
S11300200C9445000C9445000C9445000C94450038
S11300300C9445000C9445000C9445000C94450028
S11300400C9445000C9445000C9445000C94450018
S11300500C94450011241FBECFE5D8E0DEBFCDBF10
S113006010E0A0E6B0E0EEEBF0E002C005900D92E7
S1130070A036B107D9F710E0A0E6B0E001C01D92A8
S1130080A036B107E1F70C944D000C94000002C0B7
S1130090000001970097E1F70895CFE5D8E0DEBFAF
S11300A0CDBF84E08ABB17BA14BA11BA14E080E257
S11100B09EE40E9447008BB381278BBBF8CFE0
S9030000FC
